:10000000830100308A00AA28F20003088301B600A9
:100010000408B7000A08B8008A017008BA0071081D
:10002000B9008301201C2B28A3010730831203137E
:1000300023020318282823082B3E8400831300087A
:10004000F0002308243E840070088000A30A1528CD
:10005000A001DC30A20083120313A10A05302102A3
:100060000318A1011F3086042108243E8400831355
:10007000000888002908A3005528831203132A08C2
:10008000A3006428031083120313A30D0310A30D10
:10009000031083120313A30D0310A30D0310831287
:1000A0000313A30D0310A30D642883120313210867
:1000B000013A03194E28033A03194828013A031953
:1000C0004228073A03193D2883120313A31F6A2805
:1000D00087146B28871083120313231F71280714BA
:1000E000722807100130F000831203132108F10079
:1000F000F10A7C280310F00DF10B7A287008A30098
:10010000FF30A30623088605A20803198928A20345
:100110009A28831203132A083F39A300A30803195E
:100120009928A303C030AA052308AA04DC30A20042
:100130009A28A0140B11031383123A08F00039080F
:10014000F1003708840038088A0036088300F20E70
:10015000720E0900203084003630B52083010A1267
:100160008A11A92F04068001840A0406031DB228FF
:02017000003459
:100F24008301B50003178D0083168C130C148312F0
:100F34000C0803130800F000003071187007031048
:100F4400F00D0310F10CF108031908009F2F07306E
:100F5400831603139F008501860187018801890197
:100F640083128801871007108316811201118110E2
:100F7400011481118B168312A101A201A00100307A
:100F84000A128A1192270A128A11B3008B1783124C
:100F94000313B20133083202831203130318CB2F55
:100FA400B401073034020318F02F0730F100831224
:100FB400031332080A128A119D273407F000700ABD
:100FC4000A128A1192270A128A11F00034082B3E61
:100FD4008400831370088000B40AD32F8312031390
:100FE400A001A00AA00883120313031DF42FA00874
:0C0FF400831203130319F92FB20ACC2F4B
:02400E00333F3E
:10420000240080008000800080008000000000000A
:10421000C000C000C000C000C00055004000E00069
:10422000E000E000E000E000FF00C000F100F1006D
:10423000F100F100F100FF00C000FB00FB00FB00FB
:10424000FB00FB00FF00C000FF00FF00FF00FF00BD
:10425000FF00FF00CC00FF009F00FF00FF00FF00F9
:10426000FF000000FF008700FF00FF00FC00FF00D0
:104270000000FF008100FF00FF00F000FF000000D1
:10428000FF008000FF00FF00C000DF000000FF0013
:1042900080007F00FF000000CF000000FF008000D2
:1042A0001F00FF000000CC000000FF00800007009E
:1042B000FC000000CC000000FF0080000100F000C6
:1042C0000000CC000000FF0080000000C0000000E3
:1042D000C4000000FF008000000000000000C000DB
:1042E00000000000FF00800000000000300000001F
:1042F00000000000FF00800000000C000000000033
:1043000000000000FF0080000300000080000000AB
:1043100000000000FF000000C000FF00800000005F
:1043200000000000C0000000FF008000000000004E
:10433000FF00C000C000FF0080000000FF00FF0081
:10434000C300C000FF008000FF00FF00FF00CF009F
:10435000C000FF00FF00FF00FF00FF00FF00CC00D7
:10436000FC00FC00FC00FC00FC00000001008700D9
:104370008700870087008700FF00C100FC00FC0069
:10438000FC00FC00FC0000000100870087008700A3
:1043900087008700FF00C100FF00FF00FF00FF0053
:1043A000FF00FF00C200FB00FB00FB00FB00FB0066
:1043B000FF00C000F100F100F100F100F100FF008A
:1043C000C000E000E000E000E000E000FF00C0000E
:1043D000C000C000C000C000C00055004000800008
:1043E00080008000800080000000000000000000CD
:1043F00000000000000000000400000000000000B9
:00000001FF
